:020000040801F1
:10C0000000C0002089FD01087DFE01083100020802
:10C0100045000208490002084D0002080000000027
:10C020000000000000000000000000000000000010
:10C030000000000000000000000000000000000000
:10C0400000000000000000000000000000000000F0
:10C0500000000000000000000000000000000000E0
:10C0600000000000000000000000000000000000D0
:10C0700000000000000000008DC501080000000065
:10C080000000000000000000000000005100020855
:10C09000590002080000000000000000000000003D
:10C0A0000000000000000000000000000000000090
:10C0B0000000000061000208000000000000000015
:10C0C0000000000000000000000000000000000070
:10C0D0000000000000000000000000000000000060
:10C0E0000000000000000000000000000000000050
:10C0F0000000000000000000000000000000000040
:10C10000000000000000000000000000000000002F
:10C11000000000000000000000000000000000001F
:10C12000000000000000000000000000000000000F
:10C13000F0B543F22804C2F2000480EA040515F0C9
:10C140000F0F83B000F09580056815409D4240F0C8
:10C15000F180061D86EA040717F00F0F00F08880B3
:10C1600047681740BD4240F0EF8000F1080686EABC
:10C17000040717F00F0F7BD087681740BD4240F0CF
:10C18000E38000F10C0686EA040717F00F0F6FD06A
:10C19000C7681740BD4240F0D78000F1100686EA1C
:10C1A000040717F00F0F63D007691740BD4240F036
:10C1B000CB8000F1140686EA040717F00F0F57D062
:10C1C00047691740BD4240F0BF8000F1180686EA7B
:10C1D000040717F00F0F4BD087691740BD4240F09E
:10C1E000B38000F11C0686EA040717F00F0F3FD05A
:10C1F000C7691740BD4240F0A78000F1200686EADB
:10C20000040717F00F0F33D0076A1740BD4240F004
:10C210009B8000F1240686EA040717F00F0F27D051
:10C22000476A1740BD4240F08F8000F1280686EA39
:10C23000040717F00F0F1BD0876A1740BD4240F06C
:10C24000838000F12C06744014F00F0F10D0C36AE5
:10C250001A40AA4278D1002041F23854C0F60204B4
:10C2600001464FF6FF720346009401F0B3F8FEE773
:10C27000304681425DD9046814409C425AD14668D8
:10C2800016409E425ED184681440A34258D1C468CF
:10C290001440A34251D10446C0430818C0062546A5
:10C2A00040D504F11005A94243D9276917409F42A0
:10C2B0004CD1676904F1140017409F423AD1A36939
:10C2C0001340B3423BD1E3692C461340B34229D01B
:10C2D00032E027691740B74238D167691740B74243
:10C2E00028D1A3691340B34229D1E3690CF11004AA
:10C2F0001340B34220D1DCF8107010351740B7421C
:10C3000005F1040022D1DCF814701740B74211D1B6
:10C31000DCF818301340B34211D1DCF81C30134064
:10C32000B34209D11035A94205F1040004F1100C03
:10C33000CFD8084603B0F0BD28460C30FAE72846AF
:10C340000830F7E70430F5E73046F3E72846F1E731
:10C350002DE9F04F8BB0044600F50071069142F2D2
:10C360001172079248F28006C0F2030643F22805D4
:10C37000C2F2000505F582630993089615E0079956
:10C380000139079110D141F25453C0F602030093D2
:10C390000190069A02924FF0000001464FF6FF729C
:10C3A000034601F017F8FEE7044620460699089A6E
:10C3B000D5F80034FFF7BCFE05F58163D3E900AB87
:10C3C000041B4FEAA4041AEB040A4BEBE47BC3E919
:10C3D00000AB069B984200F0D18083420ED241F21E
:10C3E0008C53C0F60203009301904FF00000014609
:10C3F0004FF6FF72034600F0EDFFFEE7036813F00F
:10C400007F4F10D041F2B452C0F602020092019365
:10C41000CDF808A04FF0000001464FF6FF7203462A
:10C4200000F0D8FFFEE7D5F8102402F10A0246F228
:10C43000A8139A4208D94FF46143CEF200034FF497
:10C440008042C3F880209CE0B5F820144FEA0B121C
:10C4500042EA1A7305934FEA0A1204928AB24FF025
:10C460000003DDE90467B61847EB0307D5F810248D
:10C4700009998B1803F1120356EA070132D0AA1862
:10C4800066F07F0182F822144FEAD61848EA47681E
:10C490004FEAD7191C464FF001021FE068F07F01F8
:10C4A00004F8011F4FEAD81141EA49614FEAD91651
:10C4B0008846B14602F10102152A0FD141F2E0533C
:10C4C000C0F602030093019602914FF0000001466E
:10C4D0004FF6FF72034600F07DFFFEE758EA0901C0
:10C4E000DCD101E04FF0000202F1FF315C5C04F0AE
:10C4F0007F045C54D5F81034D318C5F810340368A1
:10C50000089A1340C5F8003405F581614FF0000228
:10C510004FF00003C1E900234FF00003A5F82034D9
:10C52000036813F0800F1FBFB5F820349BB243F0AF
:10C530000103A5F82034036813F4004F1FBFB5F8BA
:10C5400020349BB243F00203A5F82034036813F4AF
:10C55000803F1FBFB5F820349BB243F00403A5F819
:10C560002034036813F4003F3FF409AFB5F82034DA
:10C570009BB243F00803A5F8203400E7024BC3E95F
:10C5800002AB0BB0BDE8F08F38340020684620F0D5
:10C5900007018D4671B50024C4F20204266883B0F9
:10C5A00016F400460BD1256815F480452AD123687E
:10C5B0009A0411D403B0BDE871408546704700204D
:10C5C00041F21064C0F6020401464FF6FF720346C2
:10C5D000009400F0FFFEFEE71748FFF7B9FE4FF4A6
:10C5E0000053636023685B04E4D541F25C64C0F6E9
:10C5F0000204284629464FF6FF722B46009400F0AD
:10C60000E9FEFEE743F22800C2F20000FFF7A0FEB9
:10C610004FF48043636023689904CBD541F23864BA
:10C62000C0F60204304631464FF6FF72334600949E
:10C6300000F0D0FEFEE700BF2832002070B582B0C7
:10C640004FF43053C4F201034FF000041C809C806F
:10C650009C841C824FF00B021A854FF005029A85CC
:10C660001C839C834FF4A0529A819C861C874FF0B8
:10C670000200A3F8400043F22801C2F2000101F5D4
:10C6800082664FF000024FF00003C6E90223C1F8B2
:10C6900010444FF03003C4F202031C60586041F2B2
:10C6A0001002C4F201029A6041F21052C0F6020276
:10C6B000DA6043F6B1221A604FF48053C4F20103EA
:10C6C0004FF020021A614FF04403C4F202031C60D1
:10C6D0004FF400725A604FF0C8429A60D96043F23A
:10C6E000AF521A6041F28063C0F602030093204605
:10C6F00021464FF6FF72234600F06CFE4FF0040215
:10C70000CAF200024FF48873C1F2100313604FF0B5
:10C710000C02CAF20002136041F2A063C0F60203E9
:10C720000093204621464FF6FF72234600F052FE4A
:10C730004FF00803C4F202031A6822F400521A6090
:10C740004FF01C03C4F202031A6822F400521A606C
:10C7500041F2C863C0F602030093204621464FF61B
:10C76000FF72234600F036FE2346C4F202034FF464
:10C7700070425A604FF46143CEF200034FF480429E
:10C780001A6083F80E4341F2E863C0F60203009397
:10C79000204621464FF6FF72234600F01BFE02B0F2
:10C7A00070BD00BF2DE9F04FADF5757D82460D4699
:10C7B000934641F21473C0F6020300934FF0000059
:10C7C00001464FF6FF72034600F004FEDAF800401F
:10C7D000DAF80460B44208D054F8040B03689B688C
:10C7E00029465A469847A642F6D15D453DDA41F2C0
:10C7F0003073C0F602030393039B009301954FF03F
:10C80000000001464FF6FF72034600F0E3FD15F00D
:10C81000010F14BF04AE7CAE30464FF000014FF460
:10C82000F07204F0A7FCDAF80040DAF8048044451E
:10C830000BD04FF0F00954F8040B0368DF68314661
:10C840004A462B46B847A045F5D1E7F7E9FCA8B220
:10C850004FF00001E7F7DAFC30464FF0F001E7F760
:10C86000E1FC05F101055D45C6D10DF5757DBDE81D
:10C87000F08F00BF2DE9F04FADF50B7DCDF80CE04A
:10C880004FF003004FF00001E7F7E0FC41F2607366
:10C89000C0F6020300934FF050004FF032014FF406
:10C8A000FC624FF00003E7F7CFFC41F27C73C0F667
:10C8B000020300934FF0000001464FF6FF7203465B
:10C8C00000F088FD4FF48053C4F202039A6942F4E9
:10C8D00080429A614FF46053C4F2010340F2712226
:10C8E0001A8142F20C059D8140F60403C4F2010353
:10C8F0001A6822F0F00242F090021A601A6822F4DC
:10C90000706242F480621A6041F29C73C0F60203C6
:10C9100000934FF0000001464FF6FF72034600F00F
:10C9200059FD4FF024004FF00101E7F78FFC4FF065
:10C9300005004FF00001E7F789FC4FF009004FF0C8
:10C940000001E7F783FC4FF00A004FF00301E7F71F
:10C950007DFC4FF00B004FF00001E7F777FC4FF044
:10C960000C004FF00301E7F771FC41F2B873C0F619
:10C97000020300934FF0000001464FF6FF7203469A
:10C9800000F028FD4FF020000146E7F75FFC4FF074
:10C9900007004FF00001E7F759FC4FF008004FF097
:10C9A0000101E7F753FC4FF000000146E7F74EFCAA
:10C9B0004FF001004FF00001E7F748FC4FF008008E
:10C9C0004FF00001E7F744FC4FF009004FF0000181
:10C9D000E7F73EFC41F2D873C0F6020300934FF034
:10C9E000000001464FF6FF72034600F0F3FCE7F744
:10C9F00021FCE7F71FFC41F2F473C0F60203009339
:10CA00004FF0000001464FF6FF72034600F0E2FCD3
:10CA10004FF004044FF648752046E7F71BFC35EA53
:10CA20000000F9D141F61403C0F6020300934FF061
:10CA3000000001464FF6FF72034600F0CBFC4FF4B6
:10CA4000FA7001F05FF841F63803C0F60203009374
:10CA50004FF0000001464FF6FF72034600F0BAFCAB
:10CA6000FFF7ECFD41F65003C0F6020300934FF0D0
:10CA7000000001464FF6FF72034600F0ABFC20A811
:10CA8000C34901F091FA2CA84FF4C87120AA01F013
:10CA900077FD4FF0000479947A947B9441AE4FF087
:10CAA000F003009330464FF0400122464FF4C87324
:10CAB00002F0ACFD809679A880A900F0BBFB49ADDF
:10CAC000284620A92CAA02F03FFF43F6E712AA80CD
:10CAD0004FF03C03AB604FF0AA03EB608AA941F82A
:10CAE000245D06F1040000F0A5FB41F21056C0F6EB
:10CAF00002067CAB324652F8080F516803C36DAD95
:10CB000056F8100F7168B268F3680FC53069716923
:10CB100003C50DF5F7794FF096074FF0400002F08E
:10CB200081FF064620A92CAA234602F003F877606D
:10CB300039F8028FA6F80C808AA941F8206D42A826
:10CB400000F078FBB56805EBD575736803EB6505F8
:10CB50004FF01C0002F066FF06464FF032012A46F5
:10CB60004FF006036DAD03FB045301F025FF4FF0BA
:10CB7000010333734FF002037373A6F80E8083969C
:10CB800079A883A900F056FB04F10104A7F11E0760
:10CB9000042CC2D104AC20462CA94AF22012C0F2C7
:10CBA00007024FF0000302F01FF847F6EF33A380AF
:10CBB000E3804FF03203A3604FF0B403E36084944A
:10CBC00042A884A900F036FB73AC20462CA902F0E1
:10CBD000BDFC4FF0FF0376938AA941F8144D42A89B
:10CBE00000F028FB51AD28464FF000014FF0F00255
:10CBF00041F67403C0F6020301F0DEFE4FF00104BB
:10CC00008DF85441869579A886A900F013FB58AD9C
:10CC100028464FF041014FF0F00241F67C03C0F688
:10CC2000020301F0C9FE8DF870418AA941F80C5D3C
:10CC300079A800F0FFFA5FAD28464FF082014FF06F
:10CC4000F00241F68403C0F6020301F0B5FE8DF850
:10CC50008C418AA941F8085D79A800F0EBFA66AC2E
:10CC600020464FF4C3714FF0000241F67453C0F6F2
:10CC7000020301F0A1FE4FF002038DF8A5318DF8FB
:10CC8000A4318AA941F8044D79A800F0D3FA41F6FD
:10CC90008C03C0F6020300934FF0000001464FF6EC
:10CCA000FF72034600F096FB4FF0000BD8464BF2A4
:10CCB0008955C1F2F845029541F6B42AC0F6020A38
:10CCC0002CA8319901F082FA7EA87FA904F0A4F97A
:10CCD00043F22803C2F20003D3F810344FF0640289
:10CCE00002FB03F303F5425303F154034FEAD3036A
:10CCF000029DA5FB03537E9A009213A84FF03201C8
:10CD000041F6AC02C0F602024FEA132304F0EAFB3C
:10CD100066A813A901F038FE41F6D803C0F6020355
:10CD200000934FF0000001464FF6FF72034600F0FB
:10CD300051FB79A84FF000014FF4C872FFF732FDA4
:10CD400041F6F403C0F6020300934FF000000146E1
:10CD50004FF6FF72034600F03DFB4FF065054FF0C4
:10CD600000044FF00A064FF64877A14600E0C84697
:10CD7000013D00F0BC81304600F0C4FE4FF00400DD
:10CD8000E7F768FA6FEA00043C42F0D0AFE100BF79
:10CD900038340020FFF752FC41F61013C0F60203AE
:10CDA00000934FF0000001464FF6FF72034600F07B
:10CDB00011FB2CA84FF000024FF0000301F0D8FB4C
:10CDC00014F4005F00F0B68041F62813C0F60203A9
:10CDD00000934FF0000001460246034600F0FAFAC5
:10CDE00020A84FF000024FF0000300F025FF41F6AD
:10CDF0007010C0F6020000F0C9FD054641F6801330
:10CE0000C0F60203009301904FF0000001464FF678
:10CE1000FF72034600F0DEFA284600F043FC41F6BC
:10CE20009410C0F6020000F093FD41F6BC10C0F66D
:10CE3000020000F08DFD41F6D410C0F6020000F0B3
:10CE400087FD41F6F010C0F6020000F081FD41F6CA
:10CE50001020C0F6020000F07BFD41F63020C0F645
:10CE6000020000F075FD41F65020C0F6020000F00F
:10CE70006FFD41F67020C0F6020000F069FD41F63A
:10CE80008020C0F6020000F063FD41F69820C0F655
:10CE9000020000F05DFD984B38930FE0BDF8FA30CA
:10CEA0003A99C3F380020092C3F3C0020192504644
:10CEB00003F00102C3F3400300F04AFD20A838A9A3
:10CEC00000F038FF0028E9D141F6CC20C0F602007E
:10CED0003C9900F03DFD41F62813C0F60203009393
:10CEE0004FF0000001460246034600F073FA00F0DE
:10CEF0003BFC70B141F6D423C0F6020300930195C8
:10CF00004FF0000001464FF6FF72034600F062FA50
:10CF10000CE041F6EC23C0F6020300934FF0000052
:10CF200001464FF6FF72034600F054FA40F6B8305F
:10CF300000F0E8FD14F4807F5CD041F62813C0F6C1
:10CF4000020300934FF0000001460246034600F042
:10CF500041FA41F60430C0F6020000F017FD054624
:10CF600041F61433C0F60203009301904FF0000025
:10CF700001464FF6FF72034600F02CFA284600F0F7
:10CF80005FFDD0B141F62813C0F6020300934FF0C5
:10CF9000000001460246034600F01CFA41F6303319
:10CFA000C0F60203009301954FF0000001464FF6D2
:10CFB000FF72034600F00EFA18E041F62813C0F69F
:10CFC000020300934FF0000001460246034600F0C2
:10CFD00001FA41F64833C0F6020300934FF0000017
:10CFE00001464FF6FF72034600F0F4F940F6B83000
:10CFF00000F088FD14F4007F13D041F2883000F077
:10D0000081FD4FF00400E7F725F96FEA000414F4FE
:10D01000007F06D041F66030C0F60200039900F0B0
:10D02000DBFB48F2080323405C4514BF4FF0000BC4
:10D030004FF0010B002B0CBF00230BF0010353B189
:10D0400008F10108B8F1320FC8BF142513DCB8F19C
:10D050000A0F0BDC01E04FF00008B8F1020FCCBF63
:10D0600002250125B8F1050F05DD02E04FF00A05A4
:10D0700001E04FF0050514F0080F04D02CA8C5F10D
:10D08000000101F037FA14F4004F03D02CA8294610
:10D0900001F030FA319D15F11D0FB4BF00230123BB
:10D0A00013EA942304D02CA805F1FF3101F08EF887
:10D0B000022DCCBF0023012313EAD42304D02CA8D3
:10D0C00005F1010101F082F841F67C30C0F6020062
:10D0D000329904F0E9F94FF0040547F64076284606
:10D0E000E7F7B8F836EA0000F9D1A346E8E514F40A
:10D0F000804F3FF465AE4DE6081502084FF000037F
:10D100000B707047042A22D9438B03F00803002BCD
:10D110000CBF302331230B70438B03F00403002B2F
:10D120000CBF302331234B70438B03F00203002BE1
:10D130000CBF302331238B70438B03F00103002B92
:10D140000CBF30233123CB704FF000030B717047BD
:10D150002DE9F84304460E4615464368826893421B
:10D1600016D053F8042C03B11A60606800F1040370
:10D170006360A0F10402921B921005D04FEA820274
:10D18000801A314603F0A6FF2B683360BDE8F883B0
:10D19000D0F80090C9EB03034FEAA3034FF001025C
:10D1A00033B14FEA4302934288BF6FF0404804D83E
:10D1B0006FF04048424538BF90464FF00007B8F145
:10D1C000000F09D0B8F1804F01D302F021FC4FEAE3
:10D1D000880002F027FC0746C9EB06094FEAA909B7
:10D1E00007EB89032A680BB147F829202168751AD3
:10D1F000AD1004D038464FEA850203F06BFF07EB11
:10D20000850505F104096568AD1BAD1005D04846DC
:10D2100031464FEA850203F05DFF09EB8505206882
:10D2200008B102F00FFC2760656007EB8807A76074
:10D23000BDE8F88308B50A4641688368994207D07B
:10D24000136801B10B60436803F10403436008BD38
:10D25000FFF77EFF08BD00BF03680A6802600B602D
:10D26000704700BF20F0FF00704700BF08B500F115
:10D270008000FFF7F7FF08BDC0B2704708B5FFF7A1
:10D28000FBFFC0F5807008BD70B402784FF000035A
:10D290002AB34FF0000349F2F856C2F2000606F135
:10D2A00007044FF020012E2A18BF02460CD100F1CE
:10D2B0000102072B08DC03F1FF33F31803F8011F09
:10D2C000A342FBD14FF00803104610F8015BF55460
:10D2D00003F101035278002AE5D10A2B0ADC49F256
:10D2E000F852C2F200024FF02001995403F10103F9
:10D2F0000A2BFADD49F2F850C2F2000070BC704708
:10D3000070B582B001900091154664469CF80230D9
:10D310001BB101A86946FFF79FFF0198C0F30F20DA
:10D320000099C1F30F21E6F771FFE6F79DFFC5F500
:10D3300080754FEA450545F25653C5F2555383FBB8
:10D340000523A3EBE575C5F5807124884FEAC40277
:10D35000D2B24FEAC003DBB203FB05F302FB013399
:10D3600004F4FC664FEAE60600F4FC624FEAE202CF
:10D3700002FB05F206FB012204F478444FEA242460
:10D3800000F478404FEA202000FB05F504FB01552E
:10D3900002F1FF0032EA220228BF02464FEAA2222F
:10D3A00005F1FF0135EA250528BF0D464FEAE525C1
:10D3B0004FEAC52545EA421203F1FF0033EA230391
:10D3C00028BF034642EAE32080B2E6F721FF02B01D
:10D3D00070BD00BF2DE9F04385B005460E461746E7
:10D3E00098460CAB53F8042B0393094C20464FF09E
:10D3F000370104F066F881460094284631463A46E3
:10D400004346E6F721FF484605B0BDE8F08300BF7C
:10D41000049600202DE9F04788B00E4615461F46B9
:10D42000BDF84030ADF804304FF000038DF8063001
:10D430004FF0874102F0EAFE03F038F80446079007
:10D4400028464FF0874102F0E1FE03F02FF8054631
:10D45000069030464FF0874102F0D8FE03F026F8E0
:10D460000646059038464FF0874102F0CFFE03F0A4
:10D470001DF804902C1B0394861B0296002CB8BF49
:10D480006442002EB8BF7642B4420FDA07A805A95D
:10D49000FFF7E2FE06A804A9FFF7DEFE03A802A933
:10D4A000FFF7DAFE4FF001038DF80630079B069A6E
:10D4B0009A4207DA07A806A9FFF7CEFE05A804A935
:10D4C000FFF7CAFE029F4FEA0727039B97FBF3F77C
:10D4D000079E3046FFF7CAFE0446C6EB000907FB6D
:10D4E00009F909F1FF0539EA290928BFA946059B71
:10D4F00003EB292906F18000FFF7C0FE05464846E8
:10D50000FFF7B0FE06464846FFF7B8FE05FB00F2FF
:10D5100002F1FF0332EA220228BF1A460DF1040C81
:10D52000204631464FEA2222FFF7EAFE4846FFF73F
:10D53000A3FE05FB00F505F1FF0212EA250238BF44
:10D540002A460DF1040C204606F580714FEA22228E
:10D55000FFF7D6FE069D2846FFF788FE8046461B4D
:10D5600007FB06F606F1FF0336EA260628BF1E462D
:10D57000049B03EB262605F18000FFF77DFE0546A0
:10D580003046FFF76FFE82463046FFF777FE05FB19
:10D5900000F202F1FF0332EA220228BF1A460DF11F
:10D5A000040C404651464FEA2222FFF7A9FE3046BE
:10D5B000FFF762FE05FB00F505F1FF0212EA250206
:10D5C00038BF2A460DF1040C40460AF580714FEA37
:10D5D0002222FFF795FE04F1010408F1FF38A0456F
:10D5E0001FDB09EB07052846FFF73CFE06462846E9
:10D5F000FFF744FE02460DF1040C20463146FFF7CA
:10D600007FFE2846FFF738FE02460DF1040C204647
:10D6100006F58071FFF774FEED1904F58074A045DE
:10D62000E1DA08B0BDE8F087F8B50D461E4688423D
:10D630000CDC044697B2A0B23946E6F7E7FD304667
:10D64000E6F7E6FD04F10204A542F4DAF8BD00BFF6
:10D65000F8B515461E4691420CDC0C4687B238469A
:10D66000A1B2E6F7D3FD3046E6F7D2FD04F102049D
:10D67000A542F4DAF8BD00BF08B5FFF705FE014684
:10D6800049F2F853C2F2000303F1440003F5277294
:10D6900003F52973E6F7FAFDD0F1010038BF002049
:10D6A00008BD00BF10B5FFF7EFFD014649F2F85481
:10D6B000C2F2000404F1440004F5277204F5297352
:10D6C000E6F7E2FDD0F1010038BF002084F8A8029F
:10D6D0004FF00003C4F8AC32C4F8B032C4F8B4322E
:10D6E00000F0010010BD00BF08B549F2F853C2F2C6
:10D6F000000393F8A8327BB349F2F853C2F2000357
:10D70000D3F8B022991881F8440002F10102C3F85D
:10D71000B022D3F8AC1201F10101C3F8AC12B2F59A
:10D72000007F19D319464FF00003C1F8B032D1F889
:10D73000B43203F10103C1F8B43201F1440001F540
:10D740002771E6F7A7FD38B149F2F853C2F200039A
:10D750004FF0000283F8A82208BD00BF08B50846B4
:10D76000FFF7C2FF08BD00BF38B549F2F853C2F257
:10D77000000393F8A83263B349F2F853C2F20003EE
:10D78000D3F8B03263B14FF0200549F2F854C2F239
:10D7900000042846FFF7A8FFD4F8B032002BF8D1D8
:10D7A00049F2F853C2F200034FF0000283F8A822B6
:10D7B000D3F8B41203F144004FEA412103F5277274
:10D7C00003F52973E6F768FDD0F1010038BF0020AA
:10D7D00038BD4FF0000038BD2DE9F04387B006AFEB
:10D7E00004460D467B4649F2F85EC2F2000ECEF8C2
:10D7F000B8327346CEF8BC326B46CEF8C0323B46E8
:10D80000CEF8C4320EF5327E41F68836C0F60206F6
:10D810000FCEAEE80F0096E80F008EE80F004FF035
:10D820001F00E6F7F7FC4FF003004FF00001E6F7AA
:10D830000DFD41F60043C0F60203009301944FF042
:10D840000A004FF0DC014FF6FF724FF00003FFF7C4
:10D85000C1FD41F61043C0F60203009301954FF05D
:10D860000A004FF0CE014FF6FF724FF00003FFF7B2
:10D87000B1FD3C4641F62043C0F6020300930197F8
:10D880004FF00A004FF0C0014FF6FF724FF0000357
:10D89000FFF7A0FD4FF0B20541F63846C0F602068C
:10D8A0004FF00A084FF6FF790096236801936368EA
:10D8B0000293A3680393E36804934046A9B24A46DF
:10D8C0004FF00003FFF786FDA5F10E0504F11004EB
:10D8D000182DE9D141F65443C0F6020300934FF0EE
:10D8E000000001464FF6FF720346FFF773FD41F655
:10D8F0006840C0F60200FFF7D5FE4FF000554FF428
:10D900004044C2F2000415F8010BFFF7EDFEA542FA
:10D91000F9D1FFF729FF68B141F67443C0F602035D
:10D9200000934FF0000001464FF6FF720346FFF7E9
:10D9300051FD0CE041F69043C0F6020300934FF016
:10D94000000001464FF6FF720346FFF743FDFEE776
:10D950000FB430B583B006AB53F8042B49F2F8543A
:10D96000C2F20004D4F8AC5201934FF000004DF223
:10D970005D71C0F6010103F0C0FCD4F8AC02401B9D
:10D9800003B0BDE8304004B0704700BFF8B50646AC
:10D990004FF00004094D4FF00D0728463946324636
:10D9A000234603F09FFD2846FFF766FE20B104F1F1
:10D9B0000104B4F57A7FF0D10048F8BDE09800206A
:10D9C0002DE9F0014FEAC00C5FFA8CFC00F4FC6713
:10D9D0004FEAE70700F478404FEA202617494FF056
:10D9E0000002104644F23F25C0F20F0531F8023F15
:10D9F0004FEAC3085FFA88F8C8EB0C08B8F1000FCB
:10DA0000B8BFC8F1000803F4FC64A7EBE404002CE1
:10DA1000B8BF6442444403F47843A6EB2323002BAD
:10DA2000B8BF5B42E3189D42C4BF10461D4602F1D9
:10DA30000102102ADAD1BDE8F0017047A61B0208E6
:10DA40002DE9F041FFF72EFE41F68835C0F60205BC
:10DA500005F13F0405F1750514F8010FFFF744FEC9
:10DA6000AC42F9D141F68836C0F6020606F11E0432
:10DA700006F13E064FF0000734F8025F05F47840E7
:10DA80004FEA1020FFF730FE05F4FC604FEAD000AB
:10DA9000FFF72AFE4FEAC50000F0F800FFF724FE6A
:10DAA0003846FFF721FEB442E6D14FF00007B846F2
:10DAB00021E020463146E6F7A9FBE6F7D5FBFFF764
:10DAC0007FFF054604F1010080B23146E6F79EFB78
:10DAD000E6F7CAFBFFF774FF40EA0510C0B2FFF794
:10DAE00003FE04F10204A4B2B4F5C87FE1D107F14A
:10DAF0000107F02F02D04446BEB2DAE7FFF734FE4A
:10DB0000BDE8F08149F63C13C2F2000318801A46C2
:10DB100013889BB2002BFBD1704700BF08B42DE9DE
:10DB2000F04F88B002908846914611AB53F804BB81
:10DB300003934FF0000741F62813C0F60203049345
:10DB4000039B03F104030593049B00934FF0000033
:10DB5000414602460346FFF73DFCCDF800B002986F
:10DB600041464A464FF00003E6F76EFB584603F085
:10DB70001BFB059B0793039B1C684FF0000504B338
:10DB8000029B03F1100606EBC0064FF0000500945F
:10DB9000B0B241464A46BD4214BF00230123E6F716
:10DBA00053FB204603F000FB00F1020006EBC00629
:10DBB00005F10105079B03F1040207921C68002C84
:10DBC000E5D14FF06400FFF79DFF4FF0040648F2E7
:10DBD000480A3046E6F73EFB80F47E4080F4A474A9
:10DBE00014EA0A0FF5D04FF004064FF6487A304693
:10DBF000E6F730FB5045FAD14FF06400FFF782FFA3
:10DC0000002FD4BF0023012313EAD40318BF07F168
:10DC1000FF3799D114F4004F05D005F1FF35AF421D
:10DC2000B8BF013790DB14F0400F8DD0384608B0F4
:10DC3000BDE8F04F01B07047F0B589B00546164613
:10DC40001F463B4B009356EA07010FD14FF00001EE
:10DC500041604FF000024FF00003C0E90423C0E927
:10DC600006230184418480F828105EE0D0E9042373
:10DC7000964277EB03011BDA4468A4FB060104FB20
:10DC80000711D5E9062302F037FC241A84420FD984
:10DC90004FF0000169604FF000024FF00003C5E94A
:10DCA0000423C5E906232984698485F8281007E040
:10DCB00095F8283023B12B689B6928466946984718
:10DCC000D5E90623B24273EB070106DA2B685B69DC
:10DCD0002846694698470028F2D1D5E9062396429E
:10DCE00077EB030107DA2B689B692846694698475A
:10DCF0000028F2D112E095F82830B3B14FF00001BE
:10DD000069604FF000024FF00003C5E90423C5E944
:10DD100006232984698485F8281006E0D5E90623BE
:10DD2000964277EB0301E9DBE5E709B0F0BD00BF00
:10DD3000081502082DE9F00F82B00446884690F8D5
:10DD40002830002B40F09B80C36A1B6842689A42CF
:10DD50001BD300F11801D1E90001C8E90201E36A0F
:10DD6000D3E90223861841EB0307C8E90467E36A95
:10DD70001B8AA8F81A30628CA8F81820B04271EB00
:10DD80000703BCBF012384F82830D4F82C90D9F8BD
:10DD9000003062689A4257D24FF000014FF0000203
:10DDA0004FF00003CDE90023D4F804C009EB0C03C5
:10DDB000987CC2B24FF000034FF07F0A4FF0000B87
:10DDC00002EA0A0603EA0B07A1F1200306FA03F5AB
:10DDD000C1F1200226FA02F207FA01FB42EA0B0B1C
:10DDE0001BEA230B38BFAB4606FA01FADDE9002334
:10DDF00042EA0A0243EA0B03CDE900230CF10103D6
:10DE0000636001F10701C9B210F0800FCCD1D4E9F1
:10DE10000601C8E90201009D4FEA1512DDF804A0D1
:10DE200042EA0A724FEA1A13121843EB0103C8E9D7
:10DE30000423628CA8F8182005F00F03A8F81A3004
:10DE40004FF0000384F82830D8E90223C4E9042302
:10DE5000D8E90423C4E90623B8F818A0A4F820A040
:10DE6000B8F81AB0A4F822B0D8E90201D8E904231E
:10DE7000904271EB0304ACBF0020012001E04FF0A1
:10DE8000000002B0BDE8F00F704700BF2DE9F00FB1
:10DE9000436893B390F828304BB9C26A436803F1E2
:10DEA000FF334360D31893F91130002BF6DB45683C
:10DEB000C46A641904F112044FF000064FF0000721
:10DEC0004FF07F0A4FF0000B4FEAC71949EA566935
:10DED0004FEAC61814F8012D4FF0000302EA0A02B7
:10DEE00003EA0B0342EA080643EA0907013D09D0A9
:10DEF00014F9013C002B05DAE6E74FF00000BDE81D
:10DF0000F00F7047D0E90423C1E90223D0E90645A8
:10DF1000C1E90445048C0C83448C4C83C0E906237E
:10DF20004FEA161444EA07744FEA1715D1E90223A1
:10DF3000121B63EB0503C0E9042306F00F060E83F2
:10DF400046844FF0FF3303844FF0000380F82830FD
:10DF50004FF00100D3E700BF10B504464FF030008A
:10DF600001F060FD0D4B0360636843600C4B836000
:10DF7000D4E90423C0E90423D4E90623C0E9062335
:10DF8000084B8360238C0384638C438494F828308B
:10DF900080F82830E36AC36210BD00BF181D020874
:10DFA000081D02080815020830B404460A4B036035
:10DFB0004FF0000545604FF000024FF00003C0E94C
:10DFC0000423C0E9062305844584044A826080F85E
:10DFD0002850C16230BC7047181D0208081502089D
:10DFE000014B0360704700BFC01C0208014B036077
:10DFF000704700BFC01C0208014B0360704700BFA0
:10E00000C01C020810B50446024B036001F01AFD63
:10E01000204610BDC01C020810B50446024B036028
:10E0200001F010FD204610BDC01C020810B50446CA
:10E03000024B036001F006FD204610BDC01C020823
:10E0400038B505464FF0200001F0ECFC0446074BC4
:10E0500003602B685B6928462146984720B9204613
:10E0600001F0F0FC4FF00004204638BD081502080E
:10E0700030B440690028A8BF02FA00F010DAC0F1FD
:10E080000001A1F1200043FA00F4C1F1200503FAD8
:10E0900005F322FA01F21A4334EA200028BF1046A1
:10E0A00030BC70474369002BA3BF41FA03F3184605
:10E0B000C1175B42BEBF01FA03F31846C117704790
:10E0C0002DE9F04704468A46FFF7ECFFD4E90889BA
:10E0D00018EB000849EB01096568A668B5421CD039
:10E0E0002B689A45C4BF05F11804274608DC14E0E4
:10E0F00004F11804631BDB1953F8303C9A450CDD1E
:10E1000054E9022354E90401121A63EB010318EBEA
:10E11000020849EB0309A642EAD140464946BDE858
:10E12000F08700BF2DE9F84F844692469B4644682D
:10E130008568AC4204BF4FF000084FF0000926D1BB
:10E1400034E0F0E8066701F11801564577EB0B0360
:10E1500010DA0C4651E90423B21A67EB030318EBFB
:10E16000020849EB03098D42EBD11FE04FF0000894
:10E170004FF00009D4E9022392457BEB030115DB44
:10E18000564577EB0B0311DB2068BDE8F88FD4E927
:10E190000467564577EB0B01E8DA04F1180104F146
:10E1A00028004FF000084FF00009D2E752465B46C6
:10E1B000B2EB080263EB0903DCE908456046121B79
:10E1C00063EB0503FFF754FFBDE8F88F2DE9F04F2F
:10E1D0009BB006464161006803689968D6E906234A
:10E1E00088471AA99E4B41F8383D306803685B693F
:10E1F00098473046B16AFFF755FF4FF0FF324FF0B6
:10E20000FF33841841EB0305CDE90A45316901EB81
:10E21000D17130464FEA6101FFF744FFCDE90401B7
:10E220004FF0000A4FF0000BD046D9466BE0CDE925
:10E230001023DDE91023141B63EB0505DDE90A015A
:10E24000DDE90823904271EB030354DA3046F16AAA
:10E25000FFF728FFCDE90601079F4FEAD771DDE9F7
:10E260000623521843F1000359104FEA3200CDE95A
:10E270000001844275EB010108DA1AEB040A4BEB4A
:10E28000050B18EB040849EB05093CE0DDE9002328
:10E2900012EB080243EB0903CDE90223DDE9040197
:10E2A000824273EB01011DDADDE90823121B63EBE7
:10E2B0000503CDE908231AEB040A4BEB050BDDE956
:10E2C0000023DDE9084594429D4101DADDE9082398
:10E2D000DDE90601821A61EB030318EB020849EB42
:10E2E000030910E0DDE900231AEB020A4BEB030BF4
:10E2F000DDE9028907E01AEB040A4BEB050B18EB8A
:10E30000040849EB0509DDE90445A04579EB05055D
:10E3100080F2BC80306803689B690CA9984700288C
:10E3200000F0B480DDE91001DDE90E4502460B4640
:10E33000121B63EB0503CDE90823D6E906238242CD
:10E3400073EB0107FFF673AF73E74FF000024FF076
:10E350000003C6E9082341F64850C0F60200316ABE
:10E3600003F0A2F8306803689968D6E90823884763
:10E370007368B36041F65C5AC0F6020A4FF00007BA
:10E380004EE050464146C8EB040203F08DF8149766
:10E39000159716971797189719973046F16AFFF750
:10E3A00081FE4FEAD173C01841F1000149104FEAD4
:10E3B0003000DDE90E23841841EB0305CDE9164555
:10E3C000DDE91023101A63EB0101CDE91801D6E94C
:10E3D0000823944275EB030E01DACDE91623DDE93B
:10E3E0001623824273EB01041ADA3046FFF79AFED5
:10E3F0001490B468F3689C420CD034B114AD0FCDC6
:10E400000FC495E8030084E80300B36803F1180320
:10E41000B36005E006F10400214614AA00F072F989
:10E42000306803685B690CA9984700284CD0DDE987
:10E430000E89304642464B46FFF774FE33699842D8
:10E4400042DADDE91045304622462B46B2EB08029F
:10E4500063EB0903FFF70CFEB36A9842E0DD90E737
:10E460000815020851E90423DDE90E01904271EB21
:10E4700003053CDA306803685B690CA998470028FB
:10E4800035D1B368A3F11803B36030E041F678509A
:10E49000C0F60200514603F007F8DDE90423B2EBB1
:10E4A000080263EB090312EB0A0243EB0B03D6E904
:10E4B0000601821A61EB0303C6E90823002A73F1FF
:10E4C0000007BFF648AF40E7B1687368CB1A4FEA60
:10E4D000E30303EB830202EB02124FEA022012185D
:10E4E0004FEA0240121803EB4203002BBAD11BB0D3
:10E4F000BDE8F08FF8B504460D46D0E90667324610
:10E500003B46FFF70FFE41192046FFF7D9FDC4E94E
:10E51000060186EA000287EA010352EA030E16D1D9
:10E52000002D09DD4FF001024FF00003921943EB7B
:10E530000703C4E906230AE0002D08DA4FF0FF3292
:10E540004FF0FF33121843EB0103C4E90623D4E96B
:10E550000623002A73F1000105DA4FF000024FF0A4
:10E560000003C4E9062320466169FFF72FFEF8BDCA
:10E5700008B5C0E906234169FFF728FE08BD00BFC2
:10E5800010B504464FF00003036043608360C3602E
:10E590000161436101EBD1734FEA6303836201F1CF
:10E5A000030331EA210128BF19464FEAA101C162E4
:10E5B00013681B6910469847226820601AB11368D7
:10E5C0005B68104698474FF000024FF00003C4E923
:10E5D00008232046FFF7CCFF204610BD2DE9F0416F
:10E5E00006460C460B684B6082684368D31A4FEAB4
:10E5F000E30303EB830101EB01114FEA01228918C8
:10E600004FEA01428918204603EB410100F022F84D
:10E610007568D6F80880454519D02F466668A36806
:10E620009E420BD02EB10FCF0FC697E8030086E8AD
:10E630000300636803F11803636004E02046314679
:10E640002A4600F05FF805F11805A845E5D1BDE8B8
:10E65000F08100BF2DE9F04104460D464AF6AA2399
:10E66000C0F6AA23994205D941F63850C0F60200F7
:10E6700001F0C4F907688368DB1B4FEAE30303EB8F
:10E68000830202EB02124FEA022152184FEA0241C2
:10E69000521803EB42039D4232D94368DB1B4FEA19
:10E6A000E30303EB830606EB06164FEA0622B618D1
:10E6B0004FEA0642B61803EB46064FF0000835B1A4
:10E6C00005EB45004FEAC00001F0ACF980463EB1D1
:10E6D00006EB4602404639464FEAC20202F0FAFC17
:10E6E000206808B101F0AEF9C4F8008006EB4606D8
:10E6F00008EBC606666005EB450508EBC505A56099
:10E70000BDE8F0812DE9F04387B004468846914684
:10E71000476883689F4238D06D46A7F118060FCE30
:10E720000FC596E8030085E8030037B16D460FCDAD
:10E730000FC795E8030087E80300606800F118033D
:10E740006360A0F11803C8EB03034FEAE30303EB94
:10E75000830202EB02124FEA022152184FEA0241F1
:10E76000521813EB420207D002EB42024FEAC202F8
:10E77000801A414602F0AEFCB9E80F00A8E80F008D
:10E7800099E8030088E80300A4E005687F1B4FEACE
:10E79000E70707EB870303EB03134FEA03229B18FA
:10E7A0004FEA03429B1807EB43074AF6AA23C0F639
:10E7B000AA239F4205D141F24870C0F6020001F041
:10E7C0001DF94FF0010347B14FEA47039F4284BF51
:10E7D0004AF6AA26C0F6AA2606D84AF6AA26C0F6FF
:10E7E000AA26B34238BF1E464FF0000776B14AF65C
:10E7F000AA23C0F6AA239E4201D901F009F906EB2B
:10E8000046004FEAC00001F00DF90746C5EB0805C8
:10E810004FEAE50505EB850303EB03134FEA0322FB
:10E820009B184FEA03429B1805EB430505EB450592
:10E8300017EBC5051FBFB9E80F000FC599E8030026
:10E8400085E803002168C1EB08034FEAE30303EB0B
:10E85000830505EB05154FEA0522AD184FEA054281
:10E86000AD1813EB450506D005EB450238464FEAD7
:10E87000C20202F02FFC05EB450507EBC50909F1C3
:10E8800018096368C8EB03034FEAE30303EB83054E
:10E8900005EB05154FEA0522AD184FEA0542AD1804
:10E8A00013EB450507D005EB4502484641464FEAC4
:10E8B000C20202F00FFC05EB450509EBC505206817
:10E8C00008B101F0BFF82760656006EB460607EB6C
:10E8D000C607A76007B0BDE8F08300BFF8B50446DF
:10E8E0000E4685694FEAC5054168407B012808BF8F
:10E8F000A1EB650103D0022808BFC5EB01015B1A3B
:10E90000AB42B4BF0025012555EAD3753AD1A568BD
:10E91000217B012908BF073D02D009B9A5F10E05E9
:10E92000002D2FDB05F10E0191422BDC03F10702D4
:10E9300012EA230238BF1A464FEAE20261698F5C8D
:10E940004FEAE3724FEA5272991801F00701891AEF
:10E95000384689B2E5F760FC202F14BF0746002730
:10E960004FF0000306EB45053A46C7F38007217CCC
:10E970008F421CBFE189E952C2F34F0703F1020342
:10E980001C2BF1D1F8BD00BF70B504460D460846FA
:10E9900002F00AFCA06100F1010001F057F8064600
:10E9A000A269294602F1010202F070FB606966610A
:10E9B00008B101F04FF870BD38B50446084D056048
:10E9C000416082604FF00002027342734FF0FF31EA
:10E9D000C181027442611946FFF7D6FF204638BD57
:10E9E000A81D0208014B0360704700BF901D02087C
:10E9F000704700BF10B50446024B036001F022F8D7
:10EA0000204610BD901D020810B50446064B036059
:10EA100040694FF00003636108B101F01BF8034B3C
:10EA20002360204610BD00BFA81D0208901D0208EB
:10EA300010B50446074B036040694FF00003636163
:10EA400008B101F007F8044B2360204600F0FAFFFC
:10EA5000204610BDA81D0208901D02082DE9F047B0
:10EA600004468A46806B1946FFF72AFB8046894692
:10EA70004FF000052E4604F11807638E1E4365EA29
:10EA80000305ADB2D4E90A23904579EB030107DB16
:10EA9000206903685B69394698470028EDD12FE06B
:10EAA000A38A1E420CBF002201221D420CBF00237C
:10EAB00001231A4212D06368A2689A18934225DA99
:10EAC0000AEB430AA2892AF8022B03F101036168C9
:10EAD000A2688A189A42F5DCBDE8F0874AB16268FC
:10EAE000A368D31803F1FF33A4892AF81340BDE8C3
:10EAF000F0875BB16368A4892AF81340BDE8F0870A
:10EB0000D4E90A23904579EB0301C9DBBDE8F0871E
:10EB100010B50446806BFFF7D3FA02460B46206916
:10EB2000016889688847206903685B6904F11801F6
:10EB3000984710BDF8B5044617461E46114B0360B2
:10EB40004FF0000545604FF0100383604FF0FF3336
:10EB500083810B681B690846984720614FF00103C9
:10EB600003FA06F6A6824FF000024FF00003C4E954
:10EB70000823C4E90A2325866586034BA361A7639E
:10EB80002046F8BDC01D02080815020810B504464D
:10EB9000064B036000694FF00003236110B1036866
:10EBA0005B689847024B2360204610BDC01D0208D9
:10EBB000901D020810B50446084B036000694FF031
:10EBC0000003236110B103685B689847044B23601E
:10EBD000204600F037FF204610BD00BFC01D0208D0
:10EBE000901D02080000000030B40C4D05604FF687
:10EBF000FF758580C5804FF0140585604FF0DC05FA
:10EC0000C560C0E904234FF000038361C361036260
:10EC100043628362C362016330BC7047D81D02083F
:10EC20002DE9F04F83B082468B464FF44A44C3F639
:10EC30009A34A2FB040104FB0311DDE90C2301F06B
:10EC40005BFC80468946B8F57A7F79F1000009DAE5
:10EC50005046594641F6E852C0F60202434602F0D9
:10EC600041FC7FE04FF47A744FF000054FF47A7165
:10EC70003FA7D7E9006701E014461D46A4FB012326
:10EC800001FB0533904579EB030EB4BF0020012052
:10EC9000A64277EB050EB4BF002000F0010000286B
:10ECA000EAD14046494622462B4601F025FC06465D
:10ECB000092821DC4FEAE07300FB05F104FB031196
:10ECC000A6FB0423CB18B8EB020869EB03094FF04D
:10ECD0000A03A8FB030103FB091122462B4601F09E
:10ECE0000BFC00905046594641F6F052C0F6020225
:10ECF000334602F0F7FB08E05046594641F6FC5215
:10ED0000C0F60202334602F0EDFB0AEB0001C0EB55
:10ED10000B064FF47A724FF0000362406B4052EAE8
:10ED2000030008D10846314641F60062C0F60202EF
:10ED300002F0D8FB16E044F24022C0F20F024FF07E
:10ED4000000354405D4054EA05030846314607BFBE
:10ED500041F60462C0F6020241F60862C0F6020201
:10ED600002F0C0FB03B0BDE8F08F00BFAFF300803E
:10ED7000FFC99A3B000000002DE9F041C768069CDE
:10ED80002568A5F1050405F10505AB42ACBF0026D9
:10ED90000126A342D4BF002606F0010646B108466C
:10EDA0004FF000014FEA420202F0E4F9BDE8F081C1
:10EDB000A7F11007BA42A8BF3A469C4239DBE31AD2
:10EDC000C3F1050C4FEA4C0C4FEA430884681C1948
:10EDD000A24269DD4FF00007838821F8143004F166
:10EDE000010303EB0C069A42D4BF00250125B34270
:10EDF000ACBF002505F0010585B101EB440424F802
:10EE0000027F03F101039A42D4BF002501259E42EF
:10EE1000D4BF002505F00105002DF0D19A42C4BFF2
:10EE2000848821F8134003EB0804A242D4DCBDE837
:10EE3000F0819D4238DCEB1A03F10504C3F10003B5
:10EE40004FEA43074FEA440C8368E3189A422BDDEC
:10EE50004FF00008848821F81340DC19A242C4BF97
:10EE6000838821F8143004F1010303EB0C059A4266
:10EE7000D4BF00260126AB42ACBF002606F0010637
:10EE800086B101EB440424F8028F03F101039A4296
:10EE9000D4BF002601269D42D4BF002606F00106FD
:10EEA000002EF0D19A42D5DCBDE8F0812DE9F04387
:10EEB00083B00646894690461D468369C0698342F1
:10EEC00014D01A68A2F10A01A9420BDC02F10A026D
:10EED000954207DC00933046494642462B46FFF7F1
:10EEE0004BFF03E003F118039842EAD1746AB66A53
:10EEF000B4420AD02368DF682046494642462B4682
:10EF0000B84704F11C04A642F4D103B0BDE8F08375
:10EF10002DE9F04F89B0064602910392006B06F18D
:10EF20001801FFF75BFB776AB56AAF4208D03C4631
:10EF300023681B682046984704F11C04A542F7D1BA
:10EF4000B76206F1240AF269B369D31A4FEAE30300
:10EF500003EB830101EB01114FEA012289184FEA0B
:10EF600001428918504603EB410100F0A5F8B3694E
:10EF7000F269D21A4FEAE20202EB820101EB0111BF
:10EF80004FEA012009184FEA0140091802EB41023B
:10EF9000002A47D04FF00007B84606F10C0B03EBF0
:10EFA0000709DB593BB3D9E90423D9E90245D6E97E
:10EFB0000401CDE9000105A84FF00A01121B63EB23
:10EFC0000503FFF72DFE504649465A4605AB00F0B3
:10EFD0007FFAB36A4FF0010203F80F2CB36AF2888C
:10EFE00023F80E2CB06A50F81C3C9B68A0F11C0062
:10EFF0000299039A984708F10108B36907F11807C5
:10F00000F269D21A4FEAE20202EB820101EB01112E
:10F010004FEA012009184FEA0140091802EB4102AA
:10F020009045BCD309B0BDE8F08F00BFAFF30080BE
:10F0300070B506460C4B0360446A856AAC4207D043
:10F0400023681B682046984704F11C04A542F7D1A9
:10F05000706A08B100F0F6FCB06908B100F0F2FC8B
:10F06000024B3360304670BDD81D0208901D020867
:10F0700070B506460E4B0360446A856AAC4207D001
:10F0800023681B682046984704F11C04A542F7D169
:10F09000706A08B100F0D6FCB06908B100F0D2FC8B
:10F0A000044B3360304600F0CDFC304670BD00BFED
:10F0B000D81D0208901D02082DE9F84305460F46A9
:10F0C00049F24923C0F62413994205D941F6385034
:10F0D000C0F6020000F092FC06688268921B4FEABC
:10F0E000A20246F6B753CBF2DB6303FB02F399426D
:10F0F0004FD94468C6EB04094FEAA90946F6B7534D
:10F10000CBF2DB6303FB09F94FF0000831B1C1EB2F
:10F11000C1004FEA800000F085FC8046A6421CD06A
:10F1200043461D484FF000018BB1186072685A6069
:10F13000B2689A60327B1A73727B5A73F289DA81F1
:10F14000327C1A74726971615A61B2699A6103F111
:10F150001C0306F11C06B442E6D12C686E68B4426A
:10F1600007D023681B682046984704F11C04A64278
:10F17000F7D1286808B100F065FCC5F80080C9EB3C
:10F18000C90908EB89036B60C7EBC70708EB870762
:10F19000AF60BDE8F88300BFA81D02082DE9F04F5D
:10F1A0008FB004460391049205930D46436882682C
:10F1B000934200F0AA80EBB16E4A1A6053F8182C03
:10F1C0005A6053F8142C9A6013F8102C1A7313F821
:10F1D0000F2C5A7333F80E0CD88113F80C2C1A74B8
:10F1E00053F8082C4FF0000143F8081C5A6153F8FB
:10F1F000042C9A61676807F11C036360A7F11C0681
:10F200000399C1EB060A4FEAAA0A46F6B753CBF2B6
:10F21000DB6303FB0AFABAF1000F42DD02970196A5
:10F22000A7F138020092B346B04691460198331ACE
:10F2300000995B185A6802983B1A5B445A6001991E
:10F24000C1EB0905009AAD186B6AC0EB08045C4479
:10F25000636295F8283084F8283095F8293084F8CE
:10F2600029306B8D638595F82C3084F82C3056F856
:10F27000083C4FF0000046F8080C57F8080C47F817
:10F28000083C08B100F0E6FB6B6B6363A7F11C0759
:10F29000A6F11C06A9F11C09A8F11C08BAF1010A83
:10F2A000C4D107A8049A1168059B1A68189BFFF738
:10F2B00083FB089B03984360099B83609DF828307B
:10F2C00003739DF829304373BDF82A10C1819DF85E
:10F2D0002C3003740C9B4FF000020C9202464069E4
:10F2E000536108B100F0B6FB0D9B039883610EAB30
:10F2F000204A43F81C2D58694FF000030C93002856
:10F3000000F0E18000F0A6FBDDE006689B1B4FEA01
:10F31000A30246F6B753CBF2DB6303FB02F349F2D9
:10F320004922C0F62412934205D141F24870C0F63A
:10F33000020000F063FB4FF0010243B14FEA4302C9
:10F34000934284BF49F24927C0F6241706D849F2F0
:10F350004927C0F62417BA4238BF17464FF0000BB2
:10F360008FB149F24923C0F624139F4204D900F01B
:10F370004FFB00BFA81D0208C7EBC7004FEA800083
:10F3800000F050FB834603998B1B23F00303049A80
:10F390001168059802681BEB030002D0189BFFF769
:10F3A0000BFBD4F800C003998C4508BF5E4631D0F2
:10F3B00062465B46454E4FF000008BB11E605168BF
:10F3C000596091689960117B1973517B5973D18988
:10F3D000D981117C197451695061596191699961A0
:10F3E00003F11C0302F11C029542E6D10CF11C0250
:10F3F000039B9A1A4FEA920246F6B753C3F2DB63B5
:10F4000003FB02F323F0404606F10106C6EBC606F5
:10F410000BEB860606F11C0A65680398854239D015
:10F4200002465346DFF8A4904FF000080AF1140C8E
:10F43000B3B1C3F800905168596091689960117B2D
:10F440001973517B5973D189D981117C1974506911
:10F45000C2F81480991B614441F81C0C91699961B0
:10F4600003F11C0302F11C029542E1D1039B03F15D
:10F470001C02AA1A4FEA920246F6B753C3F2DB63A4
:10F4800003FB02F323F0404303F10103C3EBC30387
:10F490000AEB830A25686668B54207D02B681B68AB
:10F4A0002846984705F11C05AE42F7D1206808B1FF
:10F4B00000F0C8FAC4F800B0C4F804A0C7EBC7074E
:10F4C0000BEB8703A3600FB0BDE8F08FA81D020807
:10F4D000F0B583B004460E461546476882689742E9
:10F4E0000AD009682A6817B13846FFF765FA6368D9
:10F4F00003F11C03636005E00093394632462B4656
:10F50000FFF74CFE03B0F0BD10B442699A4211D12E
:10F51000446883689C420DDA22464FF0000301EBF9
:10F5200044018489CC5202F1020203F1040384688D
:10F530009442F6DC10BC704710B5044603691846C7
:10F54000D3E90623FEF7EEFD606110BD064A0260B6
:10F550004FF0140242604FF0DC0282604FF6FF72FF
:10F56000C2600161704700BF181E0208014B0360B2
:10F57000704700BF901D020810B50446024B03609F
:10F5800000F060FA204610BD901D0208F8B503692E
:10F59000934218DA86698E4215DDCF1AB242D4BF83
:10F5A000C3EB0206C3EB060627EAE77744688568E3
:10F5B000AC4208D054F8040B03689B6839463246C5
:10F5C0009847A542F6D1F8BD2DE9F8430446884690
:10F5D0001E460369B34217DC83699E4214DA45680C
:10F5E000D0F808904D450FD055F8040B62690168BA
:10F5F000D4F81CE02369CF6808EB4201C2EB0E028D
:10F60000F31AB847A945EFD1BDE8F88330B4074DE8
:10F6100005604FF0000545608560C560016142618D
:10F620008361029BC36130BC704700BF301E02087B
:10F6300010B50446044B0360406808B100F002FABC
:10F64000024B2360204610BD301E0208901D0208A8
:10F6500010B50446064B0360406808B100F0F2F9AB
:10F66000044B2360204600F0EDF9204610BD00BF9A
:10F67000301E0208901D02082DE9F843064689460F
:10F68000174698468469C4B1C569581B214600F0E5
:10F6900071FA214600F02EFA281880450DD1B36882
:10F6A00009EB4309BB4208DAF268934205DAB288F3
:10F6B00029F8022B03F10103F4E7BDE8F88300BF4A
:10F6C0002DE9F04F9FB0814640694FF00001FEF7F1
:10F6D000F7FC04460D46D9F814004FF4C871FEF744
:10F6E000EFFCCDE90C01D9F81000036899682246B7
:10F6F0002B468847924B0E9316AC924D0FCD0FC4FC
:10F7000095E80F0084E80F00D9F814305B69059381
:10F71000002BA3BF0523059C2341059DBEBF6B4263
:10F72000052202FA03F30A934FEAE37ECDF82CE0B8
:10F730004FF0000408944FF000044FF00005CDE9AD
:10F7400006454FF0FF344FF0FF35CDE900454FF04F
:10F750000108CDF824804AE008FA04F31E4240D0A4
:10F760002F46D5E900236FEA02006FEA030150EA51
:10F77000010E32D0DDE902ABBAEB020A6BEB030BF0
:10F780000098019900EA0103DDE9000182457BEB65
:10F790000101ACBF00220122B3F1FF3F14BF1346A9
:10F7A00042F001039BB950465946DDE9002300F0C1
:10F7B000A3FE042811DCDDE9062312EB0A0243EB69
:10F7C0000B03CDE90623089B1B18089305E0CDE940
:10F7D00006ABCDE900AB09980890DDE90223C7E943
:10F7E000002304F1010405F10805042CB4D1D9F873
:10F7F000100003685B690EA99847002800F09C8000
:10F80000DDE91045CDE90245DDE90C01844275EBE7
:10F81000010180F29180DDE90A45DDE900018442C1
:10F8200075EB0101ACBF00230123009C019D04EA9C
:10F830000502B2F1FF3F08BF43F00103002B7BD06C
:10F84000BDF85230BDF850605E40B6B216AD4FF014
:10F85000000481E7C0F10001A1F12002DDF81CE005
:10F860004EFA02F0C1F120040EFA04F4069D25FAC6
:10F8700001F3234330EA220028BF18464EFA01F173
:10F88000089A4FEAE27300F037FEC9F818001BE04F
:10F89000A0F12002069B03FA02F1C0F120041D46EC
:10F8A00023FA04F4DDF81CE00EFA00F3234305FA12
:10F8B00000F031EA220128BF1946089A4FEAE273A4
:10F8C00000F01AFEC9F81800D9F81830B3F5A02FC7
:10F8D000BCBF0023C9F81830D9F81430D3E9064565
:10F8E000D9F810000368996822462B468847D9F852
:10F8F000100003685B690EA99847DDE912ABDDE9EA
:10F90000106750465946001B61EB050122462B4605
:10F91000921B63EB0703904271EB0305D9F81400C7
:10F92000B9BF52465B4632463B46FEF7FBFBC9F881
:10F930001C001FB0BDE8F08F05981030A8D589E7EE
:10F9400008150208581E020870B5044616460A4BF0
:10F9500003604FF0FF3383804FF0000585604FF068
:10F96000F003C3600B681B69084698472061666115
:10F97000A561E561204670BD481E020810B5044629
:10F98000064B036000694FF00003236110B1036868
:10F990005B689847024B2360204610BD481E020852
:10F9A000901D020810B50446084B036000694FF033
:10F9B0000003236110B103685B689847044B236020
:10F9C000204600F03FF8204610BD00BF481E020848
:10F9D000901D020808B541F67860C0F60200714635
:10F9E000FDF7FAFE08BD00BF08B541F68C60C0F611
:10F9F00002007146FDF7F0FE08BD00BF08B541F6F4
:10FA0000A060C0F602007146FDF7E6FE08BD00BF2B
:10FA100008B541F6B460C0F602007146FDF7DCFEA1
:10FA200008BD00BF38B5754601F072FA044630B91A
:10FA300041F6C460C0F602002946FDF7CDFE20461F
:10FA400038BD00BF08B501F0D5FA08BD08B5FFF70D
:10FA5000E9FF08BD08B501F0CDFA08BD4FF0000080
:10FA6000704700BF10B40B4679B144184FF4605191
:10FA7000C4F201010A8812F0800FFBD010F8012BAC
:10FA80008A80A042F6D1184601E04FF0000010BC79
:10FA9000704700BF0B1891EA000F02D493EA000FE1
:10FAA00001D4184670474FF000407047431A91EA5E
:10FAB000000F02D593EA000F01D4184670474FF0AB
:10FAC0000040704710B50446FFF7E4FFB0F1004F67
:10FAD00003D1002CC8BF6FF0004010BD10B5044624
:10FAE000FFF7E4FFB0F1004F03D1002CC8BF6FF067
:10FAF000004010BD30B44FEAE0734FEAE17200FB02
:10FB000002F201FB0323A0FB01455D194FEAE53337
:10FB1000002C75F100020DDAB3F1FF3F18BF4FF072
:10FB2000004011D14FF0FF324FF0FF33A41845EBE6
:10FB3000030502E04FF0004033B94FEA144343EAB3
:10FB40000543C4F3C034181930BC704738B50446B7
:10FB50000D46FFF7CFFFB0F1004F09D16FEA050561
:10FB60004FEAD57585EAD475002D18BF6FF00040B7
:10FB700038BD00BFF0B404460D464FF000400029E8
:10FB800067D084EAE470A0EBE47085EAE571A1EB4C
:10FB9000E5710B0D1FBF4E0C0136B0FBF6F6A6FB50
:10FBA00001231DBF520C42EAC332C2EB0000002603
:10FBB00011F00F0F18BF112311D14FF011034FEAAD
:10FBC0001111A3F1040311F00F0F14BF0022012241
:10FBD000032BD4BF002202F00102002AEFD16FEA0A
:10FBE00003024FEAD27200280CBF002202F0010289
:10FBF00022B34FF0FF3CB0FA80F7BB42B8BF1F46BC
:10FC000000FA07F2DB1BB2FBF1F02CFA03F730EA43
:10FC100007071CD100FA03F03618B2FBF1F001FB24
:10FC2000102203F1FF3350000CBF00220122002BF1
:10FC3000B4BF002202F00102002ADCD106F101006B
:10FC40004FEA500095EA040F48BF404201E04FF0F0
:10FC50000040F0BC704700BF38B504460D46FFF7C2
:10FC600089FFB0F1004F09D16FEA05054FEAD5755C
:10FC700085EAD475002D18BF6FF0004038BD00BF75
:10FC800030B4C2F5807300FB03F301FB02F24FEACC
:10FC9000E275D41845EBE3754FEA142040EA05609D
:10FCA00030BC704730B4C2F5803300FB03F301FB76
:10FCB00002F24FEAE275D41845EBE3754FEA1440BF
:10FCC00040EA054030BC704770B44FEAE073C2F1BF
:10FCD0000006A0FB064506FB03554FEAE173A1FBB6
:10FCE000020102FB0311001941EB0501084670BC3B
:10FCF000704700BF08B541F66872C0F6020243F2D1
:10FD00000003C2F200039A4206D01A4643F22803C7
:10FD1000C2F200039A420AD343F22802C2F200025E
:10FD200049F65813C2F200039A4213D320E041F679
:10FD30006872C0F6020243F20003C2F2000343F20B
:10FD40002800C2F2000052F8041B43F8041B83424F
:10FD5000F9D3E1E743F22803C2F200034FF00001B8
:10FD600049F65812C2F2000243F8041B9342FBD337
:10FD700049F65813C2F2000318460249C91A01F0A5
:10FD800011F908BD00B00020DFF828D06B46C2F2A0
:10FD900000039D464CF20003C0F601034FF46D4290
:10FDA000CEF200029360FFF7A5FFE4F75FFAFCF7DD
:10FDB00061FDFEE700C000200928D9BF3030C0B285
:10FDC0003730C0B2704700BF70B582B00A2806D085
:10FDD00049F6F003C2F200031A683F2A1DD149F622
:10FDE000F004C2F200042368E3184FF000061E710D
:10FDF00043F20005C2F20005298804F104030093D0
:10FE00004FF00A004FF6FF723346E4F71DFA266002
:10FE10002B68A3F10E032B6008E049F6F003C2F251
:10FE200000039918087102F101021A6002B070BD56
:10FE300038B50546A1B101F1FF34285D4FEA101035
:10FE4000FFF7BAFFFFF7C0FF285D00F00F00FFF7D4
:10FE5000B3FFFFF7B9FF04F1FF34B4F1FF3FECD17A
:10FE600038BD00BF10B50446007828B1FFF7ACFFDD
:10FE700014F8010F0028F9D110BD00BF704700BF72
:10FE8000F0B583B04FF01F00E4F7C4F94FF0030062
:10FE90004FF00001E4F7DAF941F6D460C0F6020051
:10FEA000FFF7E0FF41F6F460C0F60200FFF7DAFF6B
:10FEB00049F6F004C2F2000404F144004FF00401DA
:10FEC000FFF7B6FF41F6FC60C0F60200FFF7CAFF7D
:10FED00002A840F804DD4FF00401FFF7A9FF41F646
:10FEE0000470C0F60200FFF7BDFF606C00F118005F
:10FEF0004FF00401FFF79CFF41F60C70C0F60200C2
:10FF0000FFF7B0FF606C00F114004FF00401FFF741
:10FF10008FFF41F61470C0F60200FFF7A3FF606C7C
:10FF20004FF00401FFF784FF41F62070C0F6020095
:10FF3000FFF798FF606C00F104004FF00401FFF739
:10FF400077FF41F62870C0F60200FFF78BFF606C68
:10FF500000F108004FF00401FFF76AFF41F634702A
:10FF6000C0F60200FFF77EFF606C00F10C004FF05E
:10FF70000401FFF75DFF41F63C70C0F60200FFF799
:10FF800071FF606C00F110004FF00401FFF750FFAB
:10FF900041F64470C0F60200FFF764FF4EF62C50A5
:10FFA000CEF200004FF00401FFF742FF41F650701F
:10FFB000C0F60200FFF756FF4EF62850CEF20000C2
:10FFC0004FF00401FFF734FF41F65870C0F602000D
:10FFD000FFF748FF4FF0000449F6F005C2F20005B4
:10FFE00041F6F066C0F6020641F66477C0F60207F5
:10FFF000686C00EB84004FF00401FFF719FF4FEA33
:020000040802F0
:10000000E4734FEA9373E21802F00302D31A032B4E
:100010000CBF38463046FFF725FF04F10104202CC1
:10002000E6D141F66470C0F60200FFF71BFFFEE761
:10003000EFF3088249F6F003C2F200035A64FFF7B7
:100040001FFF00BFFEE700BFFEE700BFFEE700BFE7
:1000500008B5E4F7D5F808BD08B5E4F7D3F808BD4E
:1000600010B549F6F004C2F20004A36C03F10103D9
:10007000A3644FF013004FF00001E4F7E7F8B4F881
:100080004C309BB233B1B4F84C2002F1FF3292B243
:10009000A4F84C2049F6F003C2F2000393F84E3066
:1000A0005BB149F6F003C2F2000393F84E2002F16F
:1000B000FF32D2B283F84E2010BD49F6F003C2F2EF
:1000C00000034FF0140283F84E201B6D3BB149F63C
:1000D000F003C2F200031A6D02F1FF321A6549F60D
:1000E000F003C2F20003B3F854309BB2132B0BD9C8
:1000F00049F6F003C2F20003B3F85420A2F114024F
:1001000092B2A3F8542005E04FF003004FF0000135
:10011000E4F79CF849F6F003C2F2000393F8563076
:10012000312B0BD849F6F003C2F2000393F85620A6
:1001300002F10102D2B283F856201FE049F6F00422
:10014000C2F200044FF0000384F856304FF0040070
:100150004FF00101E4F77AF8B4F8583003F10103E5
:100160009BB2A4F85830B4F85A309BB233B1B4F80B
:100170005A2002F1FF3292B2A4F85A2049F6F00355
:10018000C2F2000393F85C2002F10102D2B283F8BC
:100190005C2093F85C300B2B13D949F6F003C2F2C4
:1001A00000034FF0000283F85C2093F85D20D2F149
:1001B000010238BF002283F85D204FF0010283F86E
:1001C0005E2049F6F003C2F2000393F85F3053B1AA
:1001D00049F6F003C2F2000393F85F2002F1FF3208
:1001E000D2B283F85F2049F6F003C2F2000393F81D
:1001F000603053B149F6F003C2F2000393F8602077
:1002000002F1FF32D2B283F8602010BD4FF0FF0C34
:100210001CEAD0521EBF1CEAD15392EA0C0F93EA9B
:100220000C0F6FD01A4480EA010C400218BF5FEA3D
:1002300041211ED04FF0006343EA501043EA5111B0
:10024000A0FB01310CF00040B1F5000F3EBF4900AA
:1002500041EAD3715B0040EA010062F17F02FD2AAE
:100260001DD8B3F1004F40EBC25008BF20F0010091
:10027000704790F0000F0CF0004C08BF49024CEAA8
:10028000502040EA51207F3AC2BFD2F1FF0340EA3A
:10029000C250704740F400004FF00003013A5DDCAB
:1002A00012F1190FDCBF00F000407047C2F10002EC
:1002B000410021FA02F1C2F1200200FA02FC5FEAD9
:1002C000310040F1000053EA4C0308BF20EADC7023
:1002D000704792F0000F00F0004C02BF400010F495
:1002E000000F013AF9D040EA0C0093F0000F01F042
:1002F000004C02BF490011F4000F013BF9D041EA64
:100300000C018FE70CEAD15392EA0C0F18BF93EA65
:100310000C0F0AD030F0004C18BF31F0004CD8D18F
:1003200080EA010000F00040704790F0000F17BF16
:1003300090F0004F084691F0000F91F0004F14D05C
:1003400092EA0C0F01D142020FD193EA0C0F03D1B4
:100350004B0218BF084608D180EA010000F00040B7
:1003600040F0FE4040F40000704740F0FE4040F492
:10037000400070474FF0FF0C1CEAD0521EBF1CEA31
:10038000D15392EA0C0F93EA0C0F69D0A2EB03024F
:1003900080EA010C49024FEA402037D04FF08053E9
:1003A00043EA111143EA10130CF000408B4238BFAE
:1003B0005B0042F17D024FF4000C8B4224BF5B1ABC
:1003C00040EA0C00B3EB510F24BFA3EB510340EA0A
:1003D0005C00B3EB910F24BFA3EB910340EA9C00B8
:1003E000B3EBD10F24BFA3EBD10340EADC001B0128
:1003F00018BF5FEA1C1CE0D1FD2A3FF650AF8B42CC
:1004000040EBC25008BF20F0010070470CF0004CD8
:100410004CEA50207F32C2BFD2F1FF0340EAC25003
:10042000704740F400004FF00003013A37E792F0C4
:10043000000F00F0004C02BF400010F4000F013A22
:10044000F9D040EA0C0093F0000F01F0004C02BF1D
:10045000490011F4000F013BF9D041EA0C0195E786
:100460000CEAD15392EA0C0F08D142027FF47DAF1F
:1004700093EA0C0F7FF470AF084676E793EA0C0F0F
:1004800004D14B023FF44CAF08466EE730F0004C0D
:1004900018BF31F0004CCAD130F000427FF45CAF9D
:1004A00031F000437FF43CAF5FE700BF4FEA40020A
:1004B000B2F1FE4F0FD34FF09E03B3EB12620DD992
:1004C0004FEA002343F0004310F0004F23FA02F0FC
:1004D00018BF404270474FF00000704712F1610FA3
:1004E00001D1420205D110F0004008BF6FF000407A
:1004F00070474FF00000704773B96AB9002908BF10
:100500000028BCBF00204FF00041C4BF6FF0004185
:100510004FF0FF3000F03AB882B0EC462DE90050C1
:1005200000F006F8DDF804E002B00CBC704700BF34
:100530002DE970431E4614468046894600F028F88F
:10054000A4FB002304FB01F400FB0644E318069C13
:10055000B8EB020269EB0303C4E90023BDE8708332
:10056000F8B5144606460F461D4600F0C3F900FBD9
:1005700005F5A0FB042304FB0154E318069CB21A02
:1005800067EB0303C4E90023F8BD00BF704700BF59
:1005900000292DE9F04F1C4685B0A8BF4FF0000898
:1005A000C0F2CB80002CC0F2C2800F460E469446AB
:1005B000144605461946002B4CD1BA426BD9B2FA03
:1005C00082F353B1C3F1200117FA03F630FA01F2B6
:1005D0000CFA03F4164310FA03F54FEA14493046B7
:1005E0004946A7B200F020FB49464FEA154B824628
:1005F000304600F047FC07FB0AF34BEA014B5B4532
:100600000BD91BEB040B0AF1FF3205D25B4584BF0B
:10061000AAF1020AA34400D89246C3EB0B0B494649
:100620005846ADB200F000FB49460646584600F079
:1006300029FC07FB06F745EA0145AF4206D9731EC0
:100640002D1902D2023EAF4200D81E4646EA0A46A3
:10065000002703E0BB420CD900273E46304639460E
:10066000B8F1000F02D0404261EB410105B0BDE896
:10067000F08FB3FA83F4002C40F0B180BB422CBF62
:1006800000270127824298BF47F00107002FE4D0DE
:1006900027460126E2E722B90120114600F0C4FAFC
:1006A0000446B4FA84F3002B4DD1361B4FEA1449AB
:1006B0000127A0B202904946304600F0B5FA4946FB
:1006C0004FEA154B8246304600F0DCFB029B03FBF1
:1006D0000AF34BEA014B5B450CD91BEB040B0AF107
:1006E000FF3280F0FC805B4584BFAAF1020AA3447C
:1006F00040F2F580C3EB0B0B49465846ADB200F013
:1007000093FA49460646584600F0BCFB029A02FBA3
:1007100006F345EA0145AB4206D9721E2D1902D2F5
:10072000023EAB4200D8164646EA0A4696E75242D7
:1007300063EB43036FEA080837E7404261EB41018E
:100740004FF0FF382EE79C40C3F1200126FA01F755
:1007500025FA01F24FEA14499E404946384642EADA
:10076000060B9D4000F060FA49468246384600F08C
:1007700089FBA3B202934FEA1B4703FB0AF347EA44
:100780000146B3420BD936190AF1FF3280F0AF802F
:10079000B34284BFAAF1020A361940F2A880F61AC1
:1007A0004946304600F040FA49460746304600F0D8
:1007B00069FB02981FFA8BFC00FB07F34CEA014629
:1007C000B34208D97A1E361980F08B80B34240F2CA
:1007D0008880023F3619F61A47EA0A476BE7C4F1E8
:1007E0002003A14022FA03F927FA03F649EA010996
:1007F000A74030FA03F130464FEA194B0F435946F0
:1008000002FA04FE0397CDF808E000F00DFA59460D
:100810000746304600F036FB1FFA89F3039803FBC6
:1008200007F24FEA104A4AEA014A524507D9791EAF
:100830001AEB090A59D2524557D9023FCA44C2EBB2
:100840000A0A59465046019300F0EEF95946064609
:10085000504600F017FB0198039A00FB06F31FFABD
:1008600082FC4CEA0142934207D9711E12EB090245
:1008700039D2934237D9023E4A44029946EA0746A2
:10088000C3EB020EB3B2370C88B24FEA114C00FB37
:1008900003F900FB07F20CFB03210CFB07F301EB50
:1008A00019418A4288BF03F5803303EB1147BE45E7
:1008B00012D34FEA014E1FFA89F914BF002701270E
:1008C0000EEB090215FA04F494422CBF002707F03E
:1008D0000107002F3FF4C2AE013E0027BEE692465C
:1008E00008E7174677E70E46C7E70F46A7E79246A1
:1008F00055E700BF2DE9F04F054683B00C4617467B
:1009000080468B46002B52D18A4264D9B2FA82F3D8
:1009100053B1C3F1200401FA03F130FA04F29F400D
:1009200042EA010B00FA03F83C0C58462146BEB2DD
:1009300000F07AF921464FEA184A8146584600F0FD
:10094000A1FA06FB09F34AEA014A53450BD91AEB0F
:10095000070A09F1FF3205D2534584BFA9F1020904
:10096000BA4400D89146C3EB0A0A214650461FFA02
:1009700088F800F059F921460546504600F082FA01
:1009800006FB05F648EA0148464508D96B1E18EBF8
:10099000070880F02A81023D464540F2268145EA5B
:1009A000094500263146284603B0BDE8F08F8B424A
:1009B0005AD8B3FA83F6002E59D18B422CBF0024AB
:1009C000012482428CBF254644F00105002D40F0F1
:1009D00012812E46E6E722B90120114600F024F9E3
:1009E0000746B7FA87F3002B40F0B980E41B4FEAC3
:1009F000174B1FFA87F901265946204600F014F9D3
:100A000059464FEA184A0546204600F03BFA09FBD2
:100A100005F34AEA014A534507D96A1E1AEB070A49
:100A200002D2534500F2FD801546C3EB0A0A59462F
:100A3000504600F0F9F859460446504600F022FAB4
:100A40001FFA88F309FB04F943EA0148C14508D9B4
:100A5000631E18EB070880F0CA80023CC14540F2D3
:100A6000C68044EA05459DE7002635469AE7C6F16B
:100A70002001B34032FA01F724FA01F91F43B440D0
:100A800030FA01F348464FEA174843EA040101915E
:100A90004146B240009200F0C7F84146BCB28246DF
:100AA000484600F0EFF9019804FB0AF34FEA104BB7
:100AB0004BEA014B5B4506D91BEB070B0AF1FF32F2
:100AC000C0F0A3809246C3EB0B0B4146584600F0A2
:100AD000ABF841468146584600F0D4F9019804FB32
:100AE00009F41FFA80FC4CEA01439C4205D9DB194A
:100AF00009F1FF32C0F081809146009F49EA0A491E
:100B00001C1B1FFA89FEB8B23A0C4FEA194700FBCA
:100B10000EFC00FB07F302FB0E3102FB07F201EBB8
:100B20001C418B4288BF02F5803202EB114E7445A6
:100B300011D34FEA01411FFA8CF214BF00230123A5
:100B4000B5408E18B5422CBF002603F001064D4675
:100B5000002E3FF427AF09F1FF35002622E79F4022
:100B6000C3F1200124FA01F914FA03F24FEA174BFA
:100B700025FA01F64846594646EA020A05FA03F8FC
:100B800000F052F859460646484600F07BF91FFA35
:100B900087F94FEA1A4009FB06F340EA0144A342F1
:100BA00006D9721EE41938D2A34236D9023EE4199E
:100BB000E41A5946204600F037F8594605462046C3
:100BC00000F060F91FFA8AFC09FB05F34CEA0144C6
:100BD000A34206D96A1EE41921D2A3421FD9023DBD
:100BE000E419E41A45EA064606E71D46D7E61C4620
:100BF00044EA0545D6E60125D4E69C4284BFA9F126
:100C00000209DB193FF679AF76E75B4584BFAAF1AD
:100C1000020ABB443FF657AF54E71646C8E71546ED
:100C2000DFE7023DBA4400E74A1E08BF7047C0F044
:100C30002481884240F21681114200F01781B0FAF7
:100C400080F3B1FA81F2A2EB0303C3F11F0304A204
:100C500002EB03134FF000029F4600BFAFF300808A
:100C6000B0EBC17F00BF42EB020228BFA0EBC17016
:100C7000B0EB817F00BF42EB020228BFA0EB817086
:100C8000B0EB417F00BF42EB020228BFA0EB4170F6
:100C9000B0EB017F00BF42EB020228BFA0EB017066
:100CA000B0EBC16F00BF42EB020228BFA0EBC160F6
:100CB000B0EB816F00BF42EB020228BFA0EB816066
:100CC000B0EB416F00BF42EB020228BFA0EB4160D6
:100CD000B0EB016F00BF42EB020228BFA0EB016046
:100CE000B0EBC15F00BF42EB020228BFA0EBC150D6
:100CF000B0EB815F00BF42EB020228BFA0EB815046
:100D0000B0EB415F00BF42EB020228BFA0EB4150B5
:100D1000B0EB015F00BF42EB020228BFA0EB015025
:100D2000B0EBC14F00BF42EB020228BFA0EBC140B5
:100D3000B0EB814F00BF42EB020228BFA0EB814025
:100D4000B0EB414F00BF42EB020228BFA0EB414095
:100D5000B0EB014F00BF42EB020228BFA0EB014005
:100D6000B0EBC13F00BF42EB020228BFA0EBC13095
:100D7000B0EB813F00BF42EB020228BFA0EB813005
:100D8000B0EB413F00BF42EB020228BFA0EB413075
:100D9000B0EB013F00BF42EB020228BFA0EB0130E5
:100DA000B0EBC12F00BF42EB020228BFA0EBC12075
:100DB000B0EB812F00BF42EB020228BFA0EB8120E5
:100DC000B0EB412F00BF42EB020228BFA0EB412055
:100DD000B0EB012F00BF42EB020228BFA0EB0120C5
:100DE000B0EBC11F00BF42EB020228BFA0EBC11055
:100DF000B0EB811F00BF42EB020228BFA0EB8110C5
:100E0000B0EB411F00BF42EB020228BFA0EB411034
:100E1000B0EB011F00BF42EB020228BFA0EB0110A4
:100E2000B0EBC10F00BF42EB020228BFA0EBC10034
:100E3000B0EB810F00BF42EB020228BFA0EB8100A4
:100E4000B0EB410F00BF42EB020228BFA0EB410014
:100E5000B0EB010F00BF42EB020228BFA0EB010084
:100E6000104670470CBF012000207047B1FA81F294
:100E7000C2F11F0220FA02F0704708B14FF0FF30B4
:100E8000FFF784BB0029F8D02DE90340FFF7CCFE23
:100E9000BDE8064002FB00F3A1EB0301704700BF71
:100EA00001207047704700BFC36810B4196882689A
:100EB000012921D043F20803C2F2000319694361FA
:100EC0000161186101690123036048611368012B06
:100ED00001D010BC7047436800EB030C9445F8D177
:100EE0005168C9184160516913690B615961916872
:100EF000D2689160CA60ECE759685C188442D9D125
:100F000040689A6040185860D3601846DEE700BF1A
:100F1000F8B50546E0B143F20804C2F20004A36943
:100F2000984700283BD023691A68022A0DD01F3544
:100F30005A6825F00F05954203D80BE05A68954290
:100F400008D91B691A68022AF8D10025E369984775
:100F50002846F8BD05F12001914217D859199F681C
:100F60001E695869521B4A604FF0010E002243F877
:100F700005E0CB608F600E61486183E82400F96072
:100F800099607161016103F11005DFE75D6919691D
:100F9000002029614D61186003F11005D6E7054670
:100FA000D6E700BF172938B5044600D838BD43F24C
:100FB0000805C2F20005012202604160AB69984752
:100FC0000028F3D0EB681868022804D105E0DB683C
:100FD0001968022901D09C42F9D99868E360A060A1
:100FE0009C60A2682046D460FFF75EFFEB699847DB
:100FF00038BD00BF38B5054630B143F20804C2F22F
:101000000004A369984700B938BDA5F11000FFF7A7
:101010004BFFE069804738BD70B543F208050023F7
:10102000C2F200050360AA690B6004460E469047B1
:1010300098B12B69186802280DD0586822681118D9
:1010400021605A6830681B6990422CBF3060326062
:1010500019680229F1D1EB69984770BD10B440F6C8
:10106000A56240F6A164C0F6020443F20803C0F68C
:101070000202C2F20003002808BF2046002908BF70
:1010800011469861D96110BC704700BF70B4FAB1C5
:101090000B4613F8015B8A18C9438C18934201462A
:1010A00001F8015B04F0010412D02CB113F8014BDC
:1010B000934201F8014B0BD01D4615F8016B0C460D
:1010C00004F8016B5E786B1C4E70611C9342F3D187
:1010D00070BC7047814270B421D9F2B111F8015B44
:1010E00003468218C44303F8015B1419934204F0C9
:1010F000010412D02CB111F8014B03F8014B9342BB
:101100000BD00D4615F8016B1C4604F8016B4E78A8
:10111000691C5E70631C9342F3D170BC7047002A57
:10112000FBD08B18551E13F8016C82182B46044611
:1011300005F0010502F8016C002BEED045B1CD1889
:1011400015F8015C00EB030C013B0CF8015CE4D0EA
:10115000CA1812F801CC5A1EE31803F801CC8D18F6
:1011600015F8015C04EB020C531E0CF8015CEFD186
:10117000D3E700BF10B4AAB103468218C44303F8F2
:10118000011B1419934204F001040BD01CB103F8A5
:10119000011B934206D01C4604F8011B5970631CC6
:1011A0009342F8D110BC7047037843B1024603461E
:1011B00012F8011F01330029FAD1181A7047184696
:1011C000704700BF70B5CA79CC68012300E0534373
:1011D000B0FBF3F59542FAD200251AE0CE79B0FBC8
:1011E000F3F203FB1200B3FBF6F31DB9002A01DC96
:1011F000002BF3D1092AD6B205DD0A7A002A0CBFEA
:101200005722372200E0302202EB060C04F801CB13
:101210000135002BE2D1237070BD2DE9F041D36878
:1012200004460D461746166800E0013E13F8012BF0
:101230000AB1002EF9DC7B7903B1013EB87938B1EF
:10124000FB79102B01D1023E02E0082B08BF013EC2
:10125000397969B9B04604E020462021A84708F151
:10126000FF38B8F1000FF7DC721E26EAE676961B0F
:10127000797909B12046A847BB799BB1FB79102B3E
:101280000BD120463021A84797F808C02046BCF172
:10129000000F0CBF7821582103E0082B02D1204613
:1012A0003021A847387930B103E020463021A847E3
:1012B000013E002EF9DCFE6801E02046A84716F842
:1012C000011B0029F9D1BDE8F08143688268013330
:1012D000934243603EBF036803F8011B03607047FD
:1012E00013B50268044602A800F8011D0121FEF7AB
:1012F000B9FB6068431C63601CBD2DE9F04188B0F8
:10130000984605AB06460D4614460493A9E0013401
:10131000252940F0A48000238DF808308DF80A308C
:1013200001938DF809301A46204607E0232902D0A0
:10133000302908D101E0012200E0012310F8011B4F
:1013400004460029F2D18DF80A20A1F13002D0B272
:1013500009288DF8083022D805E00A2101FB023265
:1013600014F8011B00E00022A1F130035FFA83FCB6
:10137000BCF1090FF1D9A1F16100C3B2052B02D86C
:10138000A1F1570308E0A1F141035FFA83FCBCF12E
:10139000050F03D8A1F137030A2BDEDD01926C297A
:1013A00008BF14F8011B69291BD00DD8632941D04F
:1013B00007D8582923D054D8002956D0252950D1F0
:1013C0004DE064294DD10CE073293AD002D86F2941
:1013D00047D11FE0752902D0782942D10FE00A23B6
:1013E00019E0D8F800000A2700288DF80B7008F1E2
:1013F000040716DA2D2240428DF8092011E0A1F1F0
:1014000058001023414241EB000E8DF80B308DF84F
:101410000CE002E008238DF80B30D8F8000008F14A
:10142000040701A9FFF7CEFE3046294601AAFFF7BF
:10143000F4FE12E0304698F8001008F10407A847BF
:101440000BE0D8F8001001AA049130462946FFF7B6
:10145000E4FE05AA08F104070492B84601E030460C
:10146000A847217800297FF452AF08B0BDE8F08189
:1014700013B513460C4600220090019268460349BA
:101480002246FFF73AFF01981CBD00BFE112020897
:101490000EB403B503AA52F8041B0192FFF7E8FF4C
:1014A000BDE80C4003B070470FB407B504AA52F86A
:1014B000041B02200192FFF7DBFFBDE80E4004B0E1
:1014C00070471FB500240190039101A804490294BC
:1014D000FFF713FF019B1C70029804B010BD00BF02
:1014E000CB1202080CB407B504AB53F8042B0193DC
:1014F000FFF7E7FFBDE80E4002B0704700000000B4
:10150000000000000000000005D1010800000000FC
:101510000000200020000000E0FFFF071FF8E007A8
:10152000434828412900434828422900434828438A
:101530002900434828442900537475636B20696E61
:1015400020616C69676E6D656E74206C6F6F7020C2
:1015500020200000537475636B20696E20696E74DF
:101560006572727570742070726F63657373696EE3
:1015700067206C6F6F70206174202530386C782084
:101580002530386C78202020000000004461746110
:1015900020706F696E746572206973207061737456
:1015A00020656E64206174202530386C78202020FE
:1015B00000000000546F6F206261642C206C6F7318
:1015C000742074686520485F4C2073796E63202511
:1015D00030386C7820617420256C75200000000084
:1015E000537475636B20696E20626173652D3132AF
:1015F0003820766172696E74206C6F6F7020776925
:101600007468202530386C782530386C78200000DC
:101610004F68206E6F65733A20444D4120636861C6
:101620006E6E656C2034207472616E736665722014
:101630006572726F722100004F68206E6F65733A99
:1016400020414443206669666F206F766572666C40
:101650006F7720696E204854494600004F68206E1D
:101660006F65733A20414443206669666F206F7648
:101670006572666C6F7720696E205443494600009E
:10168000303038205265647563696E672046534D6B
:10169000432077616974737461746573202000005E
:1016A00030303920446F776E67726164696E6720ED
:1016B0004C4344207472616E736665722070726967
:1016C0006F7269747920200030313020456E61627C
:1016D0006C696E6720444D4120696E746572727545
:1016E000707420202000000030313120456E61628E
:1016F0006C696E6720636170747572652054494D22
:101700003120286E6F74207265616C6C79292020FD
:101710002000000030313520507265706172696EB2
:1017200067206472617761626C657320200000003D
:101730003031362044726177696E6720636F6C7553
:101740006D6E202564202000766563746F723A3ACE
:101750005F4D5F696E736572745F6175780000003C
:101760004C6F67696320416E616C797A65722028DD
:1017700063292032303132206A70610030303120EC
:1017800053657474696E672075702064656275674F
:101790002055534152542020200000003030322088
:1017A000436F6E6669677572696E672041444320B6
:1017B000202020200000000030303320436F6E6670
:1017C00069677572696E67204144432074696D656D
:1017D00062617365202000003030342044756D6DE7
:1017E0007920726561642066726F6D2041444320E8
:1017F000200000003030352057616974696E672021
:10180000666F72206B6579626F6172642069646CC7
:10181000652020003030362057616974696E67207A
:10182000666F722041444320746F20736574746C3A
:101830006520202020000000303037205374617272
:1018400074696E6720636170747572652020200072
:101850003031322053657474696E6720757020735F
:10186000637265656E206F626A6563747320202001
:101870000000000020434C454152200020534156B7
:101880004520000020424D50200000003031332020
:101890005374617274696E6720746865206D616944
:1018A0006E206C6F6F702020200000004361707408
:1018B000757265206275666665723A2025326C64C1
:1018C0002025252020467265652052414D3A20256D
:1018D00034642042000000003031342044726177CB
:1018E000696E672073637265656E2020202020205A
:1018F000000000003031372050726F6365737369E8
:101900006E67206B65797320202020202000000066
:101910004361707475726520726573746172746569
:1019200064202020200000002020202020202020D3
:1019300020202020202020202020202020202020A7
:101940002020202020202020202020202020202097
:101950002020202020202020202020202020202087
:101960002020202020202020202020202020200097
:101970007761766573253033642E766364000000EA
:1019800057726974696E67206461746120746F2096
:10199000257320002476657273696F6E2044534F5F
:1019A0002051756164204C6F67696320416E616CE2
:1019B000797A65722024656E640A00002474696D6A
:1019C000657363616C65203275732024656E640AEB
:1019D000000000002473636F7065206D6F64756C88
:1019E00065206C6F6769632024656E640A000000DF
:1019F0002476617220776972652031204120436826
:101A0000616E6E656C412024656E640A0000000002
:101A10002476617220776972652031204220436804
:101A2000616E6E656C422024656E640A00000000E1
:101A300024766172207769726520312043204368E3
:101A4000616E6E656C432024656E640A00000000C0
:101A500024766172207769726520312044204368C2
:101A6000616E6E656C442024656E640A000000009F
:101A700024757073636F70652024656E640A0000BE
:101A800024656E64646566696E6974696F6E73203F
:101A900024656E640A0000002464756D70766172BE
:101AA00073203041203042203043203044202465D0
:101AB0006E640A0023256C7520256441202564424C
:101AC00020256443202564440A00000023256C750A
:101AD0000A00000025732073756363657373667570
:101AE0006C6C79207772697474656E004661696CFC
:101AF000656420746F2077726974652066696C650F
:101B00002E0000006C6F676963253033642E626DB0
:101B10007000000057726974696E672073637265A4
:101B2000656E73686F7420746F2025732000000049
:101B300057726F74652025732073756363657373C3
:101B400066756C6C792100004269746D6170207754
:101B500072697465206661696C65642E000000001E
:101B6000557365722D696E69746961746564206D61
:101B7000656D6F72792064756D70000058504F5319
:101B800020256C750A0000004D617220313620322C
:101B90003031322031393A34303A323000000000EE
:101BA00000000000000000000000FFFF10841F0084
:101BB000E00700F8FF07E0FF1FF8100000040080B6
:101BC000E739000000000000424DF6BB00000000B5
:101BD0000000760000002800000090010000F000E6
:101BE0000000010004000000000080BB000070172E
:101BF000000070170000100000000000000000004E
:101C000020202020202025732020202020200000BC
:101C100043616C6C65723A202530386C78000000A6
:101C200052617720737461636B202866726F6D2038
:101C30002530386C78293A0020202530386C7820FF
:101C40002530386C78202530386C78202530386C79
:101C50007800000044756D70696E67206D656D6F6A
:101C600072792E2E2E0000006D656D6F72792E64D4
:101C70006D7000004D656D6F72792064756D7065D3
:101C80006420746F206D656D6F72792E646D7000C5
:101C90004D656D6F72792064756D70206661696C39
:101CA00065642028646973632066756C6C3F292E17
:101CB0000000000000000000000000000000000024
:101CC000E1DF01082DE00108D5F90108D5F9010887
:101CD000D5F901080000000000000000000000002D
:101CE000EDDF010819E00108D5F9010841E001081C
:101CF000D5F90108D5F90108D5F90108000000005F
:101D00000000000000000000FDD0010800000000FD
:101D10000000000000000000F9DF010805E00108F4
:101D200039DC010841E0010859DF010835DD01080F
:101D30008DDE010800000000766563746F723A3A28
:101D400072657365727665006C6566745F6564675D
:101D5000655F74696D6520256C640A004272656177
:101D60006B696E67206174202531306C64202531E9
:101D7000306C640A0000000074696D6520256C6495
:101D80000A00000000000000000000000000000049
:101D9000E5E90108F5E90108F1E90108D5F90108CB
:101DA000000000000000000009EA010831EA010813
:101DB000F1E90108DDE80108000000000000000072
:101DC0008DEB0108B5EB010811EB01085DEA010894
:101DD000000000000000000031F0010871F001086F
:101DE00011EF0108ADEE0108256C64206E73000050
:101DF000256C642E2530316C75000000256C640064
:101E000020757300206D7300207300000000000037
:101E100000000000000000006DF5010879F50108E0
:101E200039F5010809F50108000000000000000074
:101E300031F6010851F601088DF50108C9F50108D0
:101E400000000000000000007DF90108A5F901086C
:101E5000C1F6010879F60108FFFFFFFFFFFFFFFF52
:101E6000FFFFFFFFFFFFFFFFFFFFFFFFFFFFFFFF82
:101E7000FFFFFFFFFFFFFFFF432B2B3A2070757220
:101E800065207669727475616C000000432B2B3AF3
:101E9000206F7574206F662072616E6765000000A8
:101EA000432B2B3A206C656E677468206572726FE5
:101EB00072000000432B2B3A2062616420616C6C3D
:101EC0006F6300006F7574206F66206D656D6F72B3
:101ED000790000000A2020202020202020204841D6
:101EE00052444641554C54202020202020202020C0
:101EF000200000000A53503A2000000020205053D8
:101F0000503A20000A50433A2000000020204C5252
:101F10003A2000000A524547533A20723020000010
:101F20002C207231200000000A2020202020207266
:101F3000322000002C207233200000002C2072314F
:101F4000322000000A53434220484653523A2000B0
:101F500020434653523A20000A535441434B2044F5
:081F6000554D503A0A00000043
:101F6800DC00000014000000020000000000000077
:101F780008300020083000200830002008300020F9
:081F8800A10E0208A50E0208DB
:040000050801FD8968
:00000001FF
